:020000040000FA
:020000007D2859
:06000A0082070C340E34E5
:1000100011341034103411340E3480340C340E3456
:1000200010340E34013411340E3480340A348034E8
:100030000E341134113411340E3480340A348034C7
:1000400011341134113413340D3480340A348034B3
:100050000E3401340F3411340F34803480340C34B6
:100060001F340234043408341F34803400341B3409
:100070000E3404348234043408341F3480340034A1
:1000800020342034623479342034533420343534ED
:10009000203435342034573420345434003444343C
:1000A00005346D347034663475346E3467347334AB
:1000B0002D3447346C34693465346434003444344A
:1000C00005346D347034663475346E3467340034FE
:1000D00044346934663466346534723465342E349D
:1000E00000348207303431343234333434343534EC
:1000F00036343734383439342034030185018601ED
:10010000890113219A00890A13219C00890A13216D
:100110009200890A13219B008316423081008501D9
:100120000F30860083128C21483079210301B321DE
:100130000C30792101307921FA30AB214930B321DB
:10014000C03079213A30B3215B215B210130792124
:10015000FA30AB213621AD20CC20803079215930C6
:10016000B321893079211A084B21C03079216230BE
:10017000B3212D30121C2030BD21C93079211B083C
:100180004B21080006190800061DC4281A089C0007
:100190009B01F520AD200800C22006080339033C6E
:1001A000031DCC28C22006080339033C0319D228BA
:1001B0000618DC28ED20DD28F120C22006080339CE
:1001C000031DDD28C220060803390319E22806189A
:1001D000EB28F120CC28ED20CC281821F520AD20EB
:1001E00008002721F520AD20080089011A088800A1
:1001F0000721890A1C0888000721890A120888003B
:100200000721890A1B088800072136210800831668
:10021000081555308900AA308900881488180E29DD
:1002200008118312080083160814831208080800B6
:100230003F301A02031908009A0A12101C081A0209
:100240009B000318080012149B099B0A0800013048
:100250001A02031C080012109A031C081A029B00C1
:100260000318080012149B099B0A08001A089D0035
:100270003F301D0203189D168316860183121D0848
:1002800086000514000000000510860183160F305B
:100290008600831208006821140803190A307120AF
:1002A000BD2115087120BD212030BD216430BD2144
:1002B0004230BD2108001030970047309800FD30D3
:1002C0009900990B6129980B6129970B6129080006
:1002D00095009301940164301502031C7229950066
:1002E000930A6B290A301502031C08009500940A32
:1002F00072298C00F03086040C080F38860587219F
:10030000F03086040C0E0F3886058721080005158D
:1003100005110130AB2108009630AB21303086004A
:1003200087212930AB21872187212930AB2120303B
:100330008600872187218030860087210130AB210C
:100340008601872180308600872186018721F03051
:1003500086008721080090001D308F008F0BAE298A
:10036000900BAC290800910011080520003E0319EC
:100370000800BD21910FB42908008C00F0308604DC
:100380000C080F38860585158721F03086040C0E81
:0C0390000F3886058600872185110800C3
:02400E00F13F80
:084200000000000000000000B6
:00000001FF
